:10000000BCD400BCD51CBCDCCCBCD80FBCD9FFBC5C
:10001000D0F4BCD1F7BC0000DA00AD077EAD0AED2C
:10002000AD074EAD0029AC0300BCBA00BCBC00BC9F
:10003000BE20BDBA7DD0B4BCBD01BDBA7CBDBA7B0B
:10004000BDBA7001FBBCB8FFBDBA7101FB9DB99987
:10005000FFEE9DF0A49200AC00359CBDBDD27301B3
:10006000FBBDBA6CBDBA6BAD00A0BDBA7203928085
:100070001C9DBBBDBA6AAD00A0BDBA720392800DD3
:100080009DBBBDBA6A9DF08A9CF0AC003A30A0BD21
:10009000BA72ED928001E9BDBC7D985AAD00D18E57
:1000A000BDBA7101FB9DB99DBBBDBA6ABDBA7101F4
:1000B000FB9DB98E010305070B1700BDBA7101FB4B
:1000C0009DB98ED408D300C3FEC4FA05D90030D13F
:1000D0008E9CF9BDF9849CF9BDBA7001FB9CB88E69
:1000E0000000000000000000000000000000000010
:1000F0000000000000000000000000000000006799
:100100009DFF67DF00BDE86DA9020021339D028BD2
:100110009C02A90200058C9CFF8C8F9D049C02BD53
:10012000DC7308BDDC7B8C9CFF8C8FBDDC6B8C9CF6
:10013000FF8C8F9D038B9C03A90300058C9CFF8C77
:100140008F9D059C03BDDC7208BDDC7A8C9CFF8C06
:100150008FBDDC6A8C9CFF8C8F00000000000000CB
:10016000000000000000000000000000000000008F
:10017000000000000000000000000000000000007F
:10018000000000000000000000000000000000006F
:10019000000000000000000000000000000000005F
:1001A000000000000000000000000000000000004F
:1001B000000000000000000000000000000000003F
:1001C000000000000000000000000000000000002F
:1001D000000000000000000000000000000000001F
:1001E000000000000000000000000000000000000F
:1001F00000000000000000000000000000000000FF
:1002000000000000000000000000000000000000EE
:1002100000000000000000000000000000000000DE
:1002200000000000000000000000000000000000CE
:1002300000000000000000000000000000000000BE
:1002400000000000000000000000000000000000AE
:10025000000000000000000000000000000000009E
:10026000000000000000000000000000000000008E
:10027000000000000000000000000000000000007E
:10028000000000000000000000000000000000006E
:10029000000000000000000000000000000000005E
:1002A000000000000000000000000000000000004E
:1002B000000000000000000000000000000000003E
:1002C000000000000000000000000000000000002E
:1002D000000000000000000000000000000000001E
:1002E000000000000000000000000000000000000E
:1002F00000000000000000000000000000000000FE
:10030000DD6FAD00BB9202AC07BE9280F39410A5E6
:10031000525456585A5C5E60626466686A6C6E70CD
:10032000727476787A7C7E80828486888A8C8E90BD
:10033000929496989A9C9EA0A2A4A6A8AAACAEB0AD
:10034000B2B4B6B8BABCBEC0C2C4C6C8CACCCED09D
:10035000D2D423D623D623D623E123E723ED23F5D6
:1003600023F823FB24062411241723D623D6242084
:10037000242F243E24492454245F246A2475248095
:10038000248B249924B024C724D224E024F7250EFA
:1003900025192524252F253A25452550255B256E31
:1003A00025772582258D2598259B259E25A125C865
:1003B00025D025D825E025E825F025F82600260BB0
:1003C000261C262D263825D0263B26462657265F76
:1003D0002670267826D0AC03D99801AD00D1AC03A5
:1003E00000AD06D8AC0300AD0709AC03009800AD22
:1003F00000D1AC0300AC0712AC07439808AD00D1A4
:10040000BD0079AC03009809AD00D1BD0069AC0313
:1004100000BD0068AC0300AD17E6AD00D1AC030031
:100420009803BDDC879CDC980EAD00D1AC0300982E
:10043000FCBDDC859CDC980FAD00D1AC0300AD1E8B
:10044000B39810AD00D1AC0300AD1EBB9811AD0048
:10045000D1AC0300AD1EA19812AD00D1AC0300AD2C
:100460001EA99813AD00D1AC0300AD1E5F9814AD6A
:1004700000D1AC0300AD1E2C9815AD00D1AC03002B
:10048000AD1E849816AD00D1AC0300AD1004AD10C4
:10049000009817AD00D1AC0300BC02A0BC04A0BD05
:1004A000E87CBDEF78AD10009818AD00D1AC03002A
:1004B000BC0240BC0440BDE87CBDEF78AD100098A4
:1004C00019AD00D1AC0300AD1004981AAD00D1AC49
:1004D0000300AD101AAD1016981BAD00D1AC03008F
:1004E000BC03A0BC05A0BDE87CBDEF78AD1016989C
:1004F0001CAD00D1AC0300BC0340BC0540BDE87C92
:10050000BDEF78AD1016981DAD00D1AC0300AD1055
:100510001A981EAD00D1AC0300BDD078981FAD0075
:10052000D1AC0300BDD0689820AD00D1AC0300BDB4
:10053000DC6D9821AD00D1AC0300BDDC7D9822AD0F
:1005400000D1AC0300BDDC6C9823AD00D1AC03003E
:10055000BDDC7C9824AD00D1AC03009825AD00D162
:10056000AD00BB67AD17F48CAD00D1AC0300AD1787
:10057000BAAD00D1AC0300AD17C19827AD00D1AC26
:100580000300AD102C9828AD00D1AC0300AD105C79
:100590009829AD00D1AC0300AC1ECFAC123CAC131B
:1005A000E69DF9AD00D1D9009CFF67DF00BD007565
:1005B00025B9BD007625B925C2BD006EBD006DAD63
:1005C0001EC58C9CFFAC0300982EAD00D1AC145A14
:1005D000982FAD00D1AC15EC9830AD00D1AC16B170
:1005E0009831AD00D1AC17039802AD00D1AC030037
:1005F0009DF7AD00D1AC03009DF6AD00D1AC03007A
:10060000AD10879DFAAD00D1AC0300BDFA6DBDFA07
:100610006EBDFA7C9836AD00D1AC0300BDFA7DBD4D
:10062000FA6EBDFA6C9837AD00D1AC0300AD1E4731
:100630009838AD00D1AC0300AC137EAD1063983B8D
:10064000AD00D1AC0300BDFA6DBDFA7EBDFA6C9869
:100650003CAD00D1AC03009DD7AD00D1AC0300BDD3
:10066000FA6DBDFA7EBDFA6C983EAD00D1AC0300C8
:10067000983FAD00D1AC10FF9840AD00D1BDFA74E9
:10068000AC1241BDFA7219AD00BB9CF79DF7AD00ED
:10069000D1AD00BB9CF69DF6AD00D1D900AC128F58
:1006A000AD00BBBDF7B9AC1249AD00D1AD00BBBDCB
:1006B000F6B9AC1253AD00D1AD00BB98FEAD00D180
:1006C000AD00BBBDFA6AD9009DFBAD00D1AC030003
:1006D00098FEAD00D8AC0300BDEF6BBDD67003AC87
:1006E00007099801AD00D1BDBA7109BDEF7317BDFF
:1006F000D670F412AD00BB9203E8920503AC03D9A7
:100700009805AD00D18EAD00BBAD074E9800AD0091
:10071000D18E9806AD00D1BDEF6BBD0078AD00BBAA
:10072000990404AD0709F69206E8990304AD06D8CA
:10073000EC9207AC07439902AC03D99DF6AD00D10A
:10074000AC07BE9807AD00D1BD0068AC0300BDD0BA
:1007500068D5B89803BDDC879CDCBDDC7CBDDC6C57
:10076000BDD774F698FCBDDC859CDCBDDC7CBDDCB3
:100770006CAD09AAAD09AABD006ABDD0788EBDD006
:1007800068D5B8BDDC7CBDDC6CBDD774F6BDDC7C47
:10079000BDDC6CAD09AAAD09AAD105D0649FDC7C93
:1007A0006C7C6C7C6C7C6C7C6C7C6C7C6C7C6C7C09
:1007B0006C7C6CC0EAC1E4BD006ABDD0788EBD001F
:1007C00070069DF6AD00D10DBDEF73AC0966BDD6C8
:1007D0007003AC09669FDCDC076DBDBA7101FB9D3F
:1007E000B99CF5BD00727DBDF5707D7C6CBDD77385
:1007F000AC092EBD0072AC08F09DD7B26DBDF5718D
:100800007D7C6C9DD7B29803BDDC879CDC6DBDF50B
:10081000727D7C6C9DD7B26DBDF5737D7C6C9DD770
:10082000B26DBDF5747D7C6C9DD7B26DBDF5757DE7
:100830007C6C9DD7B26DBDF5767D7C6C9DD7B26D1D
:10084000BDF5777D7C6CD7009FF7BD077178BD083B
:100850007179BD09717ABD0A717BBD0B717CBD0CCC
:10086000717DBD0D717EBDD7717F9DF79CB89DD701
:10087000B29FDC7C98FCBDDC859CDC6C7C6CD6007B
:100880009FF6BD077078BD087079BD09707ABD0A02
:10089000707BBD0B707CBD0C707DBD0D707EBD0E80
:1008A000707F9DF6BD00700107BDBA7001FB9CB85A
:1008B000D8009FF8BD077278BD087279BD09727AB9
:1008C000BD0A727BBD0B727CBD0C727DBD0D727E4C
:1008D000BD0E727FD0F0D10F9DF8BDF0859CF09DCC
:1008E000D0BDF185BDF0879CD09DF89CD8AC0300AD
:1008F0009803BDDC879CDCBDDC7DBDDC7CBDDC6C95
:10090000BDD774F398FCBDDC859CDCBDDC7CBDDC14
:100910006CBD006AD5B8AD09AABDF77701F69DF7A1
:100920009CB89DF6BDBA7001FB9CB8AC0300BD003D
:100930007ABDDC7D9803BDDC879CDC7C6C7C6C7CA8
:100940006C7C6C7C6C7C6C7C6C7C6C7C6CD6FFD71F
:10095000FF9DF79CB89DF6BD00700107BDBA700100
:10096000FB9CB8AC0300BDD068AD00BB9CF5980300
:10097000BDDC879CDCBDDC7CBDDC6CBDD774F6982F
:10098000FCBDDC859CDCBDDC7CBDDC6CBD006AADE7
:1009900009AABDEF6BBDD0789DF7AD00D19DF6BD26
:1009A00000700103AD00D1AC03009FF69A009A00DD
:1009B0009E00BDDC6D9FF570BDDC7D9FDC7C186CFE
:1009C0007C6C7C6C7C6C7C6C7C6C7C6C7C6C7C6CE7
:1009D0007C6CD6FFD7FF8E6CBDD773E49803BDDC6B
:1009E000879CDC9DD79FF66001789FF76002789F17
:1009F000F8600478BDDC6D9FF571BDDC7D9FDC7C0B
:100A00006C9DD79FF66001799FF76002799FF8602F
:100A10000479BDDC6D9FF572BDDC7D9FDC7C6C9D37
:100A2000D79FF660017A9FF760027A9FF860047A98
:100A3000BDDC6D9FF573BDDC7D9FDC7C6C9DD79F1D
:100A4000F660017B9FF760027B9FF860047BBDDC52
:100A50006D9FF574BDDC7D9FDC7C6C9DD79FF6603F
:100A6000017C9FF760027C9FF860047CBDDC6D9F79
:100A7000F575BDDC7D9FDC7C6C9DD79FF660017DAC
:100A80009FF760027D9FF860047DBDDC6D9FF57669
:100A9000BDDC7D9FDC7C6C9DD79FF660017E9FF75F
:100AA00060027E9FF860047EBDDC6D9FF577BDDC43
:100AB0007D9FDC7C6C9DD79FF660017F9FF7600275
:100AC0007F9FF860047F98FCBDDC859CDC9FDC7C0C
:100AD0006C7C6CD0F0D10F9DF8BDF0859CF09DD062
:100AE000BDF185BDF0879CD09DF89CD88EBC0F00D1
:100AF000D5B8AD0BE8D5B8AD0BE8D5B8AD0BE8D59A
:100B0000B8AD0BE8D5BCAD0BE8D5B0AD0BE8D5550D
:100B1000AD0BE8D59DAD0BE8D5B0AD0BE8AD0BE85E
:100B2000D5A4AD0BE8AD0BE89DF69CFBAD0BE898AA
:100B300055BDFBB9AC0B77D5BCAD0BE8D5B0AD0B53
:100B4000E8D5AAAD0BE8D59DAD0BE8D5B0AD0BE867
:100B5000AD0BE8D5A4AD0BE8AD0BE89DF69CFBAD65
:100B60000BE898AABDFBB90FBC0F04BDFA6DBDFA26
:100B70007EBDFA6CAC0BE7D5BCAD0BE8D594AD0BE4
:100B8000E8D555AD0BE8D59DAD0BE8D594AD0BE898
:100B9000AD0BE8D5A4AD0BE8AD0BE89DF69CFBAD25
:100BA0000BE89855BDFBB9AC0BE7D5BCAD0BE8D550
:100BB00094AD0BE8D5AAAD0BE8D59DAD0BE8D59467
:100BC000AD0BE8AD0BE8D5A4AD0BE8AD0BE89DF699
:100BD0009CFBAD0BE898AABDFBB90CBC0F03BDFA9A
:100BE0006DBDFA7EBDFA6C8E9FDCDC079DF598FC2E
:100BF000BDDC859CDC6DBDF5707D7C6C9DD7B26DD8
:100C0000BDF5717D7C6C9DD7B26DBDF5727D7C6C40
:100C10009DD7B26DBDF5737D7C6C9DD7B26DBDF572
:100C2000747D7C6C9DD7B26DBDF5757D7C6C9DD758
:100C3000B26DBDF5767D7C6C9DD7B26DBDF5777DCF
:100C40007C6CD7009FF7BD077178BD087179BD092D
:100C5000717ABD0A717BBD0B717CBD0C717DBD0DC0
:100C6000717EBDD7717F9DD7B29FDC7C6C9803BD30
:100C7000DC879CDC7C6CD6009FF6BD077078BD08D5
:100C80007079BD09707ABD0A707BBD0B707CBD0C9C
:100C9000707DBD0D707EBD0E707FD8009FF8BD07C2
:100CA0007278BD087279BD09727ABD0A727BBD0B7C
:100CB000727CBD0C727DBD0D727EBD0E727FD0F058
:100CC000D10F9DF8BDF0859CF09DD0BDF185BDF0A4
:100CD000879CD09DF89CD88E00000000000000008A
:100CE0000000000000000000000000000000000004
:100CF00000000000000000000000000000000000F4
:100D000000000000000000000000000000000000E3
:100D100000000000000000000000000000000000D3
:10100000BDDC6B8EA903000106BDEF68BDE86CBCBA
:101010000200BDDC7B8EBDDC6A8EA902000106BD2C
:10102000EF68BDE86CBC0300BDDC7A8EBCD400BCAC
:10103000D51CBCDCCCBCD800BCD9F0BCD004BCD125
:10104000079CFF67DF00BD006BBD006CBD006DBD80
:10105000006EBD006FBDFA6A8C9CFF8EAD1EC5BDD3
:10106000FA6A8EAD1EC5AD1004AD101ADA00BCD4FC
:1010700000BCD51CBCDCCCBCD80FBCD9FFBCD0F4A8
:10108000BCD1F7AD074E8EBCD400BCD51CBCDCCCAB
:10109000BCD80FBCD9FFBCD0F4BCD1F7BC0000DA7F
:1010A00000AD074EAD102CBDFA68BDFA69BDDC6E0F
:1010B000BDDC7FBDD169BDD069BDD47AD064C0FE2E
:1010C000BDD776BDFA789800AD17F49DD995F09C00
:1010D000D99DDA950F9CFB9DD1950F9CD19DD29502
:1010E000F0BDFB8795F092F0BDFA79BDD46ABDDC06
:1010F0006FBDDC6EBDD179BDD069D07FC0FE8EAD35
:1011000000BB9CF79DF7AD00D1AD00BB9CF69DF6F2
:10111000AD00D1AD00BB9CF29DF2AD00D1AD00BBE6
:101120009CF19DF1AD00D1AD00BB9CF09DF0AD00F8
:10113000D19DF2679DF1679DF067D900BDFA7422D9
:1011400001BDFA762149AC03D9DF00BD006CBD00BA
:101150006DBD006BBD007EBD006FAD1B088C9CF0AB
:101160008C9CF18C9CF2AD1B19AD179CA9F78013D8
:10117000AD1B19BDF0B921B3AD179CAD11D49900C9
:10118000EB21A2A9F600E9BDD07CAD1B88AD179C70
:10119000AD1B88BDF0B9AC11B3AD179CAD11D4999E
:1011A00000EEAD1EC5AD00BBBD006E98FFAD00D119
:1011B000AC03009CFBAD1EC5AD17ABBD006EAD0012
:1011C000BB9CFF67DF00BDFA7A8C9CFF98FCAD00EA
:1011D000D1AC03009DF18B9CF1990021E69DF28B2F
:1011E0009CF2BDBA71129DF1990021F59DF2990012
:1011F00021F598008E98FF8EAD00BB9DF7AD00D114
:10120000E5AD1DE78C9CF08C9CF18C9CF2AD192B0C
:10121000AD179CAD192BBDF0B90AAD179CAD11D41B
:101220009900F00AAD17ABAD00BB98FC2233AD00BE
:10123000BB98FFAD00D1AD1E25AC0300982BAD00CF
:10124000D1BDFA722269AD00BB9CF79DF7AD00D10C
:10125000AD00BB9CF69DF6AD00D1D900BDFA74225D
:10126000B7BDFA76228FAC03D9AD00BBBDF7B9226A
:1012700049AD00D1AD00BBBDF6B92253AD00D1AD33
:1012800000BBBDFA6AD9009DFBAD00D1AC0300A93B
:10129000F780AC1359DF00BD007422B1BD007CBDE6
:1012A000006DBD006BBD006EBD006FAD1A17AD1BAC
:1012B00019AD179CAC03009DF799F0AC134D9DF64A
:1012C0009901AC134D98809CF798019CF698809CEE
:1012D000F5AD1E25AD1E0B9DEF67BDEF68AD190B7B
:1012E0009900AC13378C9CEFAD00BB992C233D9833
:1012F000009CF7987E9CF6AD192BAD179CAD192B71
:101300009DFBAD00D1AD179CAD00BB992C2345AD25
:10131000192B9DFBAD00D198809CF798019CF69805
:10132000009CF59DEF67BDEF68AD190B9900AC030C
:10133000D98C9CEFAC03008C9CEFAD00BB98FFAD4B
:1013400000D1AD00BB98FFAD00D1AC0300AD1DF1E5
:10135000AD192BAD179CAC0300DF00BD00752372E7
:10136000BD007DBD006CBD006BBD006EBD006FADEE
:101370001A17BDD07CAD1B88AD179CAC0300983903
:10138000AD00D1AD00BB9CF79DF7AD00D1AD00BB6A
:101390009CF69DF6AD00D1D900BDFA74AC13DABD50
:1013A000FA76AC13A8AC03D9DF00BD007623C8BD24
:1013B000007EBD006BBD006DBD006CBD006FAD1A41
:1013C00017A9F78009AD1B19AD179CAC0300BDD060
:1013D0007CAD1B88AD179CAC0300AD1DE7AD192B90
:1013E000AD179CAC0300BDFA742404BDFA7623F358
:1013F000AC03D9A9F7802409AD1B19AD00D1AD17F5
:101400009CAC0300AD192B23FBAD1B8823FBAD1E49
:101410000B5FAA9CF59DEF67BDEF689DFE67AD1958
:101420000B92000D8C9CFE8C9CEFAD00BB980224AF
:10143000468C9CFE8C9CEFBDBA7116AD179CC124E6
:1014400012AD00BB9801AD00D1DF00AD1E25AC038D
:1014500000AD00BB9800AD00D1E1AD174C92000388
:10146000AC0300BDFA74240EBDFA76246D9DF167BD
:10147000DF00BD00732489BD007BBD006CBD006D25
:10148000BD006EBD006FAD1AF78C9CF1DF015FAA45
:101490009CF59DEF67BDEF689DFE67A9F78024DD91
:1014A000AD1CF79200158C9CFE8C9CEFAD00BBAD83
:1014B0001B199CFBBDFA7A980224CC8C9CFE8C9C58
:1014C000EFAD179CC1248FAD00BB9801AD00D1DFFB
:1014D00000AC0300AD00BB9800AD00D1E49DF699CF
:1014E00020259ABDF57524EA259ABDD07C9CF595FA
:1014F000209CF5BDD969BDD869BDD0789FDC6DBD94
:10150000F6707D6CBDF5707CBDD068BDD0786DBDCA
:10151000F6717D6CBDF5717CBDD068BDD0786DBDB8
:10152000F6727D6CBDF5727CBDD068BDD0786DBDA6
:10153000F6737D6CBDF5737CBDD068BDD0786DBD94
:10154000F6747D6CBDF5747CBDD068BDD0786DBD82
:10155000F6757D6CBDF5757CBDD068BDD0786DBD70
:10156000F6767D6CBDF5767CBDD068BDD0786DBD5E
:10157000F6777D6CBDF5777CBDD068BDD078BDD0E9
:1015800068BDD078BDD068B8BDD87AD22DC2FEB8BB
:10159000BDD86AB8B8B8980024A3BDD07CAD1C3DB6
:1015A00024A3AD1DF1AD192BAD179C5FAA9CF59D31
:1015B000FE67AD192BBDF5820D8C9CFEAD17ABAD52
:1015C00000BB980225D88C9CFEBDBA7116AD179C45
:1015D000C125ACAD00BB9801AD00D1DF00AD1E252B
:1015E000AC0300AD00BB9800AD00D1E1AD174C924B
:1015F0000003AC0300BDFA7425A2BDFA762602AC46
:1016000003D9DF00BD0077261FBD007FBD006BBD85
:10161000006DBD006CBD006EAD1A17AD1B19B8ADE5
:10162000179CDF015FAA9CF59DFE67AD1B19BDF5F8
:10163000821A9CFB8C9CFEAD17ABAD00BBAD1EC5EA
:10164000DF00BD006FBDFA7A9802265E8C9CFEBD5D
:10165000BA7113AD179CC12625AD00BB9801AD0032
:10166000D1DF00AC0300AD00BB9800AD00D1E4AD0C
:101670001DE7AD192BAD179CAD192B92FF0AAD17C5
:10168000ABAD00BB9802269FAD179C9DF69901E873
:10169000BDBA71149DF799102678AD00BB9801ADC5
:1016A00000D1AD1E25AC0300AD00BB9800AD00D14C
:1016B000E3D600D700BDFA74266FBDFA7626C2AC19
:1016C00003D9AD1EC5AD1B08AD1B19AD179CAD1BD5
:1016D00019920007AD00BB980226F1AD179C9DF64C
:1016E0009900EBBDBA71139DF79910E2AD00BB985C
:1016F00001AD00D1AD1EC5AC0300AD00BB9800AD7F
:1017000000D1E4D600D700BDFA76270CAD1A17AD8C
:101710001B19AD179CAD1B1997DF92FF07AD00BBDE
:101720009802273AAD179C9DF69900E9BDBA71134E
:101730009DF79910E0AD00BB9801AD00D1AD1EC57D
:10174000AC0300AD00BB9800AD00D1E4AD00BB9C84
:10175000F79DF7AD00D1AD00BB9CF69DF6AD00D175
:10176000AD00BB9CF09DF09CF19DF0AD00D1DF0180
:101770005FD900AD00BBA6AA9CF9BDF9849CF9C055
:10178000F29DF9AD00D1AD00BB9200089800AD000C
:10179000D198FF8E9800AD00D198008E9DF68A9C5E
:1017A000F699FF27AA9DF78A9CF78E9DF68B9CF6EB
:1017B000990027B99DF78B9CF78EAD17C1AD17E641
:1017C0008E9DD8970F9CD89DD995F09CD99DD89582
:1017D000F09CD89DD097F09CD09DD1950F9CD19D29
:1017E000D0950F9CD08E9DDA950F9CFB9DD295F0E5
:1017F000BDFB878E9CFBAD17FF9DFBAD180D8E9D2D
:10180000D9970F9CD998F0BDD1879CD18E9CFB9D18
:10181000D895F09CD89DFB950FBDD8879CD89DD0BE
:10182000950F9CD09DFB95F0BDD0879CD08EBDD8E8
:1018300078BDD9789FD07F9FD868BDF570786BBD93
:10184000F7707B9FD06DBDF6707D7C6C9FD868BDB6
:10185000F571786BBDF7717B9FD06DBDF6717D7CA6
:101860006C9FD868BDF572786BBDF7727B9FD06DA9
:10187000BDF6727D7C6C9FD868BDF573786BBDF743
:10188000737B9FD06DBDF6737D7C6C9FD868BDF572
:1018900074786BBDF7747B9FD06DBDF6747D7C6CE6
:1018A0009FD868BDF575786BBDF7757B9FD06DBD12
:1018B000F6757D7C6C9FD868BDF576786BBDF77644
:1018C0007B9FD06DBDF6767D7C6C9FD868BDF5772B
:1018D000786BBDF7777B9FD06DBDF6777D7C6C6EA6
:1018E0007E8E9FD09803BDDC879CDC6E7E6E7EBDB5
:1018F000FE84BDFE84BDFE84BDFE8498FC98FCBDC4
:10190000DC859CDC9FD06E7E6E7E8ED014AD182E52
:10191000AD18E2AD182EAD192BBDF58205C0EE98BD
:10192000FF8EAD182EAD18E298008EBDD868BDD9D7
:10193000689FD06F9FFB68BDDA70789FD86BBDF74A
:10194000707B9FD06DBDF6707D7C6C9FFB69BDDAAE
:1019500070799FD86BBDF7717B9FD06DBDF6717D9F
:101960007C6C9FFB6ABDDA707A9FD86BBDF7727B87
:101970009FD06DBDF6727D7C6C9FFB6BBDDA707B7A
:101980009FD86BBDF7737B9FD06DBDF6737D7C6C6C
:101990009FFB6CBDDA707C9FD86BBDF7747B9FD0CA
:1019A0006DBDF6747D7C6C9FFB6DBDDA707D9FD83C
:1019B0006BBDF7757B9FD06DBDF6757D7C6C9FFB15
:1019C0006EBDDA707E9FD86BBDF7767B9FD06DBD04
:1019D000F6767D7C6C9FFB6FBDDA707F9FD86BBD08
:1019E000F7777B9FD06DBDF6777D7C6C6E7E7F9D9B
:1019F000FB8EBDD969BDD869BDDC6DBDD97ABDD8B6
:101A00006ABDD97BBDD86BBDD17CBDD06CBDDC6C53
:101A1000BDD178BDD0688EAD1EC5AD19F2AD1E47E3
:101A20009DF1679DF267D206D064C02A2AC22A2897
:101A3000BDDC7CAD1EA1AD1EB3B8B8B8BDDC6CD0AA
:101A4000202A48C02A482A53BDD078BDD068BDD7C7
:101A5000762A43D0202A5CC02A5C2A69BDD078BD92
:101A6000D068BDD7762A692A5C9DF79CF29DF69CCA
:101A7000F19DF292802ADB9DF199002A8998019CC0
:101A8000F19DF299002AA32ADBD00ABDD078BDD0FF
:101A900068C02A8B9DF18B9CF199012A899DF29255
:101AA000002ADBD00ABDD078BDD068C02AA59DF23F
:101AB0008B9CF298FF9CF1BDBA712ABE2A89AD00B9
:101AC000BBBD00740FBD00750BBD0076079800AD5F
:101AD00000D12A8998FDAD00D82A89A9F78011BDC7
:101AE000007505BD00740108AD00BB98FEAD00D8BF
:101AF0008C9CF28C9CF18EAD1EC5AD19F2AD1E5FB3
:101B0000BDDC6DBDDC6C2A20AD1EC5AD19F2AD1E6D
:101B10002CBDDC6DBDDC6C2A20BDD969BDD869BD8A
:101B2000D078BDD068BDD078BDD0689FFB68BDDAE5
:101B30007178BDD078BDD06869BDDA7179BDD078D3
:101B4000BDD0686ABDDA717ABDD078BDD0686BBD92
:101B5000DA717BBDD078BDD0686CBDDA717CBDD048
:101B600078BDD0686DBDDA717DBDD078BDD0686EAE
:101B7000BDDA717EBDD078BDD0686FBDDA717FBD32
:101B8000D078BDD0689DFB8EBDD969BDD869BDD068
:101B9000789FDC6DBDF6707DBDD068BDD0789FDCD0
:101BA0006DBDF6717DBDD0689FFB68BDDA7178BDF3
:101BB000D0789FDC6DBDF6727DBDD0689FFB69BD9E
:101BC000DA7179BDD0789FDC6DBDF6737DBDD068CC
:101BD0009FFB6ABDDA717ABDD0789FDC6DBDF6746B
:101BE0007DBDD0689FFB6BBDDA717BBDD0789FDC7B
:101BF0006DBDF6757DBDD0689FFB6CBDDA717CBD97
:101C0000D0789FDC6DBDF6767DBDD0689FFB6DBD45
:101C1000DA717DBDD0789FDC6DBDF6777DBDD06873
:101C20009FFB6EBDDA717EBDD078BDD0689FFB6F23
:101C3000BDDA717FBDD078BDD0689DFB8EBDD969FE
:101C4000BDD869BDD0789FDC6DBDF6707D6CBDF5EB
:101C5000707CBDD068BDD0786DBDF6717D6CBDF572
:101C6000717CBDD068BDD0786DBDF6727D6CBDF560
:101C7000727CBDD068BDD0786DBDF6737D6CBDF54E
:101C8000737CBDD068BDD0786DBDF6747D6CBDF53C
:101C9000747CBDD068BDD0786DBDF6757D6CBDF52A
:101CA000757CBDD068BDD0786DBDF6767D6CBDF518
:101CB000767CBDD068BDD0786DBDF6777D6CBDF506
:101CC000777CBDD068BDD078BDD068BDD078BDD0A0
:101CD00068B8D018BDD87AD207C2FEBDD86AB8B8E5
:101CE000B8BDDA7105C0ED98FF8EBDD87AD21FC29B
:101CF000FEBDD86A98008EBDDC6DBDD97BBDD86BAA
:101D0000BDD969BDD869BDD0789FDC6CBDF5707C4C
:101D1000BDD068BDD0786CBDF5717CBDD068BDD03C
:101D2000786CBDF5727CBDD068BDD0786CBDF573A4
:101D30007CBDD068BDD0786CBDF5747CBDD068BD6D
:101D4000D0786CBDF5757CBDD068BDD0786CBDF524
:101D5000767CBDD068BDD0786CBDF5777CBDD06891
:101D6000BDD078BDD068BDD078BDD068B8D018BD22
:101D7000D87AD207C2FEBDD86AB8B8B8BDDA710544
:101D8000C0ED98FF8EBDD87AD21FC2FEBDD86A982A
:101D9000008E9DD895F09CD89DD0950F9CD09DD954
:101DA000970F9CD998F0BDD1879CD198FCBDDC855C
:101DB0009CDCBDDC6FBDDC7EBDD169BDD069BDD40E
:101DC0007AD064C0FEBDD07FBDD87ABDD07EBDD0F4
:101DD0007CBDD07DBDD87BBDD878AD1EB3BDD06CE9
:101DE000BDD06EBDD07E8EAD1D92BDD46DBDD57DF6
:101DF0008EAD1D92BDD56DBDDC6EBDDC7FBDD169E4
:101E0000BDD069BDD47AD064C0FE8EAD1D92BDD563
:101E10006DBDD179BDD069BDDC7EBDDC7FBDD47A1E
:101E2000D064C0FE8EAD1EBBAD1E848EBDD46DBD14
:101E3000D57DBDDC6FBDDC7EBDD169BDD069BDD4B3
:101E40007AD064C0FE2E78BDD56DBDDC6EBDDC7F62
:101E5000BDD169BDD069BDD47AD064C0FE2E78BD35
:101E6000D56DBDD179BDD069BDDC7EBDDC7FBDD473
:101E70007AD064C0FE2E78B8BDFA762E83BDDC7CA5
:101E8000BDDC7D8EBDDC6CBDDC6DBDD46ABDDC6FA0
:101E9000BDDC6EBDD179BDD069D07FC0FEBDD56D32
:101EA0008EBDD47CD064C0FE8EBDD46CD0FFA4A403
:101EB000C0FC8EBDD47BD064C0FE8EBDD46BD0FF81
:101EC000A4A4C0FC8EAD1EBBAD1EA9AD1E848EADFC
:101ED00000BB920003AC03D9AD00BB920003AC037E
:101EE000D9982AAD00C39800AD00C39800AD00C3D7
:101EF000AD00BB920003AC03D99801AD00CC9810A3
:101F0000AD00C3980AAD00C39832AD00C39833AD9D
:101F100000C39801AD00C39800AD00C39800AD00A8
:101F2000C39800AD00C39800AD00C3980DAD00C3C9
:101F30009D0FAD00C39800AD00C39800AD00C398DD
:101F400000AD00C39800AD00C39800AD00C3980079
:101F5000AD00C39CF99CF4AD00BB920303AC03D964
:101F6000AD00BBAD00BBBDF4B9AC03D99800AD006A
:101F7000D1AC0300000000000000000000000000E1
:101F80000000000000000000000000000000000051
:101F90000000000000000000000000000000000041
:101FA0000000000000000000000000000000000031
:101FB0000000000000000000000000000000000021
:101FC0000000000000000000000000000000000011
:101FD0000000000000000000000000000000000001
:101FE00000000000000000000000000000000000F1
:101FF000000000000000000000000000000000FFE2
:1020000000000000000000000000000000000000D0
:1020100000000000000000000000000000000000C0
:1020200000000000000000000000000000000000B0
:1020300000000000000000000000000000000000A0
:00000001FF
